:020000040000FA
:0400000000000528CF
:08000800142800008316031305
:1000100088018C01831203138801C0308B000430E7
:10002000970001309000E6288E018F010C11090025
:10003000F930F0000000F00B1A280800F100182039
:10004000F10B1F28080008151820081118200800B7
:10005000F500F0398800F418881423201820F50ED4
:100060007508F0398800F418881423201820080037
:1000700064301E20F030F40030308800232005303A
:100080001E20232018202320081223202830282077
:1000900008302820013028200630282080302820F1
:1000A0000C30282008001508A1001608A000063012
:1000B0000310A1070318A00AA201A301A401A5012E
:1000C000A60110300314A10203186E28A008031D16
:1000D0006D2810300310A1077C28A00327300314DB
:1000E000A002031C7528A20A612810300310A10782
:1000F0000318A00A2730A007E8300314A102031850
:100100008928A008031D8828E8300310A107972834
:10011000A00303300314A002031C9028A30A7C2828
:10012000E8300310A1070318A00A0330A0076430C9
:100130000314A1020318A428A008031DA3286430F7
:100140000310A107A628A003A40A97280A300314C5
:10015000A102031CAD28A50AA628A1072108A60014
:100160000800F41454302820203028203D30282066
:1001700020302820A208031DC928A308031DCC286D
:10018000A408031DCF28A508031DD228A608031D17
:10019000D52830302207282030302307282030305F
:1001A0002407282030302507282030302607282033
:1001B0002030282075302820733028202030282037
:1001C00020302820F41080302820080038208316A2
:1001D00003130C15831203130C115320B120ED28C7
:02400E00313748
:00000001FF
